:1000000000000320D1010000D51700008D1700006B
:100010008D1700008D1700008D1700008D17000050
:100020008D1700008D1700008D170000D5170000F8
:10003000D51700008D1700008D1F000091200000D3
:10004000D5170000D5170000D5170000D517000000
:10005000D5170000D5170000D5170000D5170000F0
:10006000D5170000D5170000D5170000D5170000E0
:10007000D5170000D5170000D5170000D5170000D0
:10008000D5170000D5170000D5170000D5170000C0
:10009000D5170000D5170000D5170000D5170000B0
:1000A000D5170000D5170000D5170000D5170000A0
:1000B000D5170000D5170000D51700000D18000057
:1000C000D517000039190000D5170000651A000087
:1000D000D51700005D1B0000D5170000D5170000E4
:1000E000D5170000D5170000D5170000D517000060
:1000F000D5170000D5170000D5170000D517000050
:10010000D5170000D5170000D5170000D51700003F
:10011000D51700002D090000D5170000D5170000E5
:10012000D5170000D5170000D5170000D51700001F
:10013000D5170000D5170000D5170000D51700000F
:10014000D5170000D5170000551C0000D51700007A
:10015000D5170000D5170000D5170000D5170000EF
:10016000D5170000D5170000D5170000D5170000DF
:10017000D5170000D5170000D5170000D5170000CF
:10018000D5170000D5170000D5170000D5170000BF
:10019000D5170000D51700004D1D0000D517000031
:1001A000D5170000D5170000D5170000D51700009F
:1001B000D5170000D5170000D5170000D51700008F
:1001C000D5170000D5170000D5170000D51700007F
:1001D000594B4CF2205210B51A804DF628121A8055
:1001E00000BF00BF01F0FAFA544B4FF030621A60C2
:1001F000534A9A60534ADA60534B4FF470021A60C4
:10020000524B534A1A60534B1A78110703D51A7888
:1002100042F008021A70504B5049AA221A70504AF4
:10022000504B8B4204D252F8040F43F8040BF8E70A
:100230004D4B4E4900228B4202D243F8042BFAE781
:100240004B494C4A002352F8230041F82300013364
:10025000742BF8D1484B494A802103F8011B934283
:10026000FBD1474B424A1A60464B8A221A70A3F5CB
:10027000805324225A70A0221A709A799207FCD5D2
:100280009A79D406FCD4404A937903F00C03082BE6
:100290003D4BF9D101221A7148225A719A79900680
:1002A000FCD5394A9179384B4906FBD5374A38494C
:1002B00011600221516020221A709A7902F00C021A
:1002C0000C2AFAD1334B344A1A60344A344C13683E
:1002D00013F4807303D123604FF4A8531360314BA0
:1002E0004BF67F321A6000225A60072243F8042C32
:1002F0002D4AC3F80C2D62B600F09EF92368DA0788
:1003000005D52A4800F02CF9294B2A4A1A602A4BB5
:100310001B785B0609D5264C264B22689A4204D1ED
:10032000224800F01DF90023236001F0EDFE01F0EA
:100330005BFA01F051F9FEE70E20054030800440E1
:10034000823F04000100002B88ED00E0002008E05F
:100350000300008502D0074000E00740600CFF1F4B
:10036000E42400003007FF1F600CFF1F9C10FF1FDC
:100370000002FF1F0000000000E400E064E400E071
:1003800008ED00E000500640004006404480044074
:100390000000131104800440C010050010D0034079
:1003A00014D0034014E000E000002020D7C39A5D81
:1003B0001CE00340A5C3945A00F00740FFFFFFFF75
:1003C000FFFFFFFFFFFFFFFFFFFFFFFFFFFFFFFF3D
:1003D000FFFFFFFFFFFFFFFFFFFFFFFFFFFFFFFF2D
:1003E000FFFFFFFFFFFFFFFFFFFFFFFFFFFFFFFF1D
:1003F000FFFFFFFFFFFFFFFFFFFFFFFFFFFFFFFF0D
:10040000FFFFFFFFFFFFFFFFFFFFFFFFDEF9FFFF23
:1004100010B5054C237833B9044B13B10448AFF33E
:1004200000800123237010BD600CFF1F000000003E
:10043000E8240000084B10B51BB108490848AFF389
:1004400000800848036803B910BD074B002BFBD0A0
:10045000BDE81040184700BF00000000640CFF1FFB
:10046000E8240000600CFF1F0000000001210D20A7
:1004700000F08EB808B501210D2000F083F84FF48C
:100480007A7000F08BF80D20002100F07BF84FF41B
:100490007A70BDE8084000F081B800BF10B4114B7D
:1004A00053F8302092F8804234B1012379B182F8B8
:1004B00080305DF8044B704703EBC0035B681A683B
:1004C00051B922F002021A605DF8044B704782F8BD
:1004D00000315DF8044B704742F003021A605DF88A
:1004E000044B7047442200001C4A02EBC003012960
:1004F0005B6811D004291BD052F83000002280F82C
:10050000802229B1022920D0032922D01A60704705
:100510004FF480721A60704752F830004FF4A272A4
:1005200080F880121A601A6822F020021A60704760
:1005300052F830104FF4A272012081F880021A6044
:100540001A6842F020021A60704740F203121A60E3
:1005500070474FF481721A60704700BF4422000058
:1005600030B4054B054D064C002210211A602A605C
:100570002060196030BC704714D0034004D00340A1
:1005800000D003403F2801D8FFF788BF704700BF65
:100590003F2801D8FFF7A8BF704700BF2DE9F843F7
:1005A000054672B6204F214B214A1B683C681268F1
:1005B00062B6520102D5322B88BF013495B3C3F520
:1005C0003B431C4EDFF86490DFF864807F334FF4C8
:1005D0007A72A6FB031302FB04F404EB531472B605
:1005E000D9F800103A68D8F800E062B6C1F53B438C
:1005F0007F33A6FB03031EF0806FC4EB53134FF44D
:100600007A7002D0322988BF013200FB0233B3F581
:100610007A7F04D3013D05D004F57A74DFE700F05A
:10062000E3FFDCE7BDE8F8837C0CFF1F18E000E087
:1006300004ED00E0ABAAAAAAF8B54E4B4E48DFF88D
:100640005CC14E4C4E49DFF858E14E4E4E4D4F4F77
:100650004FF000621A604FF080521A604FF0005263
:100660001A604FF080421A604FF000421A60002278
:10067000026028234BF6FF70CCF80000CEF8003063
:1006800023600EF5012E0B6033602B6006F500260B
:100690003B6005F50025A36207F500278B6204F592
:1006A000012401F5012106F6E87605F6E87507F55F
:1006B0007F6710310EF1100E203433602B60CEF8BE
:1006C00000303B600B602360314CBB618B610921C2
:1006D0002160A7F5002704F58054203F08343A60D4
:1006E0002060BB60E36047F8041C04F5FD2407F5B7
:1006F000FE27043704F2FC7422603860A360FB60BC
:1007000044F8041C083404F6FC74C7F8FC2F20607D
:10071000A4F5E124A4F2DC7433602B60C7F8F81F61
:1007200021681C4841F40071216001681A4C0EF5E3
:100730007F4E0EF1E80E07F5883706F5803605F591
:10074000803541F000710160CEF8002047F6FF715E
:100750000822396033602B60226000F0A7FF192067
:10076000FFF71CFF00F026FE40F21310BDE8F84032
:10077000FFF714BF04E100E004800340148003404D
:100780001C800340248003402C80034034800340BD
:10079000008003400480044000900C400880034027
:1007A0000C800340431E032B14D872B60A4951F83B
:1007B000230068B170B4094C058834F813204668EA
:1007C00041F82360521B24F8132062B670BC7047B6
:1007D00062B6704700207047D80CFF1F9410FF1FAF
:1007E00030B472B62B4A13781D0706D52A4B196A06
:1007F000002936D0996A002941D053781C0706D5C4
:10080000254B196C00293ED0996C002939D093787A
:10081000190705D5204B196E002936D0996E89B17C
:10082000D3781B0707D51C4BD3F880207AB3D3F8B5
:10083000882011213AB162B6184B00221A7030BCE0
:1008400000F052BE0D21154C154D227843F8315061
:1008500003EBC1030830013A5860227062B630BC25
:10086000704704220D4C0F4D217843F8325003EBB2
:10087000C20308304A1E5860227062B6EFE70521B5
:10088000E1E70921DFE70822ECE70C22EAE7102282
:10089000E8E700BF442400000000FF1F550DFF1FC4
:1008A000C800400088004000431E032B1DD81B4A8F
:1008B000400140F0100030B4104472B6184CE25CB5
:1008C000032A1BD8DFE802F00212151703220D8855
:1008D000E25410F0080F14BFC823882343EA0543ED
:1008E00008310360416062B630BC704708300222B4
:1008F000EDE70522EBE708300422E8E7094A52F861
:10090000230038B1084A52F82300416042F823100E
:1009100062B6E9E742F82310034AF7E70000FF1F39
:10092000640DFF1F2C0DFF1F3C0DFF1F2DE9F04F25
:10093000DFF814B3DFF814A387B044E0AC4F4FEAFC
:10094000930807EBC809013ED9F8042003F0080317
:10095000F6B2A2F1080003F0FF04002B40F0FF8084
:1009600057F838301B0C99B222F8081C002B00F005
:10097000ED80A04B22F8064C42F8044C53F8262098
:10098000002A00F0CD819C4D55F8263058609B4CD4
:1009900045F8260034F81630194424F8161000F0F3
:1009A00083FD002800F0C081954A964B19F0080F8E
:1009B00000F1080018BF1346C9F8040047F83830A2
:1009C00008238BF800309BF80040E4B265071AD585
:1009D0008D4B1B78A3B18D490A7802F0FF0322B139
:1009E000013BDBB20B7003B900BE89490A7802F003
:1009F000FF032AB1013BDBB20B70002B00F06681D4
:100A000004238BF8003004F0080303F0FF02002BEE
:100A100000F0C9809AF80030DBB21E098ED19A0826
:100A2000DFF8CC9159F8321009EBC200C1F3830111
:100A3000013940680C2900F28580DFE801F07A7AFC
:100A40008383838383834683838307000168714D97
:100A50004068714F714E6860296088B240F28161D0
:100A60000024674B49F832304FF0010E88423C6059
:100A7000C9F81040C9F8184086F800E05C4A00F256
:100A8000E780B0F5D06F80F01B82B0F5817F00F079
:100A9000D98100F26981802800F02A82822840F002
:100AA000D781A98801F07F01042900F2D1815C4837
:100AB0005C4A890008441470547001788C0740F136
:100AC000608382F800E0022173E1534F3A682AB351
:100AD000554B524E554819883478057840298E4632
:100AE00045F0020828BF4FF0400E002C84F00104AE
:100AF0003470CEEB01010CBF8824C82409EBC80672
:100B000089B285F0010544EA0E447260198049F803
:100B1000384072440570002965D03A603D4B1A8810
:100B2000B2F5A06F0ED100219A785970404B1A701F
:100B300008E038493F4C0D68A54200F098803049E4
:100B400049F832103C4A0123137039E72C4A2D4BE7
:100B500019F0080F18BF134647F8383030E700F097
:100B6000C3FC364A364952F82630002B00F0E380A9
:100B700058688C5D42F8260003F10802C9F8042089
:100B8000032C05D8DFE804F02C02292602228A551E
:100B90001A8819F0080F0CBF8823C82343EA0243C0
:100BA00047F838300CE7E00700F19380210600F1A8
:100BB000D180A20706D5234A234913780220DBB24D
:100BC00013700870E30602D51F4B10221A7007B08D
:100BD000BDE8F08F04228A55DAE705228A55D7E767
:100BE00003228A55D4E7BEF1400F18BF002294E7D4
:100BF0000000FF1FD80CFF1F840CFF1F9410FF1F65
:100C0000C800400088004000600DFF1FE90CFF1F76
:100C1000740DFF1F4C0DFF1F800CFF1FE80CFF1F02
:100C2000C0200740580DFF1F940CFF1F540DFF1FDD
:100C30009820074021090003942007402C0DFF1F36
:100C4000640DFF1F88200740802007409020074048
:100C5000B0F5106F00F07C8140F2A38040F62112C5
:100C6000904240F07B82A54A012313706AE74C68EA
:100C7000A3498C427FF463AF0178A9297FF45FAF69
:100C8000417845297FF45BAF8178C2297FF457AF63
:100C9000C1786B297FF453AF9A489B4E0178347822
:100CA00081F00105002C41F0020105700CBF882085
:100CB000C82084F0010449F8310009EBC1019348D0
:100CC0003470002505244D60047038E700F064FCA2
:100CD00096E68F4B89488B491A614FF0020E80F8D7
:100CE00000E08C4F0A708C49196099608B4E8C4DD6
:100CF0008C4C9A610D213970FF213170DFF84CE284
:100D000029702270884D894A8EF800109F2701248F
:100D100006F8047C5D600470DA6007B0BDE8F08F0F
:100D200043F82600824D32E6824A47F838001378AD
:100D30000133137044E68B5D032B00F2BA8001A2ED
:100D400052F823F0C1090000C10900009D0D000008
:100D5000970D00006F49724B80220D2008701A70A9
:100D6000A2077FF52FAF26E740F20232904240F013
:100D7000ED81AA8802F07F02042A69D86D88002DCF
:100D800066D16449CDF804E0920011440A7842F03B
:100D900002020A70C1E101238B5511E600238B5535
:100DA0000EE6B0F5086F53D16349644A09781170B3
:100DB0007146ED888D4280F0E88252480478402DDB
:100DC000AE4644F0020C28BF4FF0400E02EB0E037B
:100DD00009EBCC01029301234A604FEA0E48CEEBA7
:100DE000050101930025C82242EA080384F00102AC
:100DF00049F83C3035700270DFF814C1424BDFF81F
:100E0000048149BBBEF1400F7FF42DAF42F0020CCC
:100E100009EBCC03029ADFF8F8E05A608DBB0D04B1
:100E200045F088059DF804304EF83C500A44337074
:100E30000470134640297FF416AF0021404A3B60FE
:100E4000118010E7AA8802F07F02042A40F28B8109
:100E5000304A0F23137006E74029D7D942F0020227
:100E60000CEBC200029E4660BDB19DF804503548AF
:100E70001D703346403988F8004040334CF832004A
:100E8000DCE79DF8043033700D04029B047045F0DC
:100E9000C8050B444EF83C50CCE79DF804501D703B
:100EA000029B1D4888F80040403940334CF832001E
:100EB000C4E719F0080F0CBF022303238B557FE50D
:100EC00021494A68002AC3D06C88B5F804E003E0E1
:100ED0000C314A68002ABBD00B88A342F8D14B885A
:100EE0007345F5D1240A032C0CBF1178098960E7FA
:100EF000124A0221147054705BE700BF942007402F
:100F000001000400540DFF1FE80CFF1FE90CFF1F38
:100F10000000FF1FC02007408800400088200740D5
:100F20008020074098200740980CFF1FEC0CFF1F03
:100F3000840CFF1F550DFF1F600DFF1F580DFF1F75
:100F4000940CFF1FC8004000482400008C2007407C
:100F5000B248116AAC7804700C0600F19881D9F897
:100F60002820AF49100600F1DB81D9F83020AC49C8
:100F7000120600F1D081D9F83820A949130600F1F2
:100F8000C581D9F84020A649150600F1BA81D9F8E3
:100F90004820A349140600F1AF81D9F85020A04998
:100FA000100600F1A481D9F858209D49120600F1DD
:100FB0009981D9F860209A49130600F18E81D9F8F9
:100FC00068209749150600F18381D9F8702094496B
:100FD000140600F17881D9F878209149100600F1C3
:100FE0006D81D9F880208E49120600F16181D9F80F
:100FF00088208B49130600F15581D9F89020884943
:10100000150600F14981D9F898208549140600F1A8
:10101000FF808448844A854901908548854D864CE7
:10102000049700230596029580460F4616461D46F6
:101030000394306828B1446800F056FA2046002C2A
:10104000F9D100233360029B38681A46002342F826
:10105000253028B1446800F047FA2046002CF9D129
:1010600000223A60019A98F800301146002241F8B7
:10107000042B039A0191023B4FF0000122F8151056
:10108000032B07D8DFE803F05D025D024FF0010398
:1010900088F800300135042D06F1040607F1040735
:1010A00008F10108C5D1654C654D2278654B049F58
:1010B000059E0021100729701A7000F19280624984
:1010C00062780A700021C9F83010C9F83810110789
:1010D000DFF84C816ED4A2785C49DFF844810A7055
:1010E00000211207C9F85010C9F858104BD4E27803
:1010F00057494B4C0A7013074FF00001C9F87010A4
:10110000C9F8781000F1AE8033780193002283F0A3
:101110000105C9F89020C9F898200021029188465D
:101120008E460A464B48047844F0020C09EBCC0387
:101130000393019B002B039B5A600CBF8822C8229B
:1011400052E64FF0000388F80030A3E7B0F5A06F37
:101150007FF47EAE012300250193DEE740F62122D5
:101160009042F7D074E66D88002D7FF471AE3A4955
:10117000CDF804E0920011440A7822F002020A70CD
:10118000CBE7022115E600F08FF9002800F0EB8094
:101190000830324AC8F86400C8F8602000F084F9CA
:1011A000002800F0DA8008302D4AC9F86C00C9F830
:1011B00068209CE700F078F9002800F0E080083013
:1011C000264AC8F84400C8F8402000F06DF900280D
:1011D00000F0CF800830224AC9F84C00C9F84820F6
:1011E00079E700F061F9002800F0A58008301B4A7B
:1011F000C9F82400C9F8202000F056F9002800F0B2
:1012000094800830164AC9F82C00C9F8282056E7FF
:10121000D1F89C00083800F067F9FAE6600DFF1F6E
:101220000000FF1F3C0DFF1FD80CFF1F2C0DFF1FE0
:10123000640DFF1F840CFF1F9410FF1F4424000047
:10124000550DFF1FC4200740C8200740CC20074091
:10125000D0200740540DFF1FC020074088004000E9
:10126000C800400000F020F9002870D008304F4A34
:10127000C4F88400C4F8802000F016F9002860D07B
:1012800008304B4AC9F88C00C9F888203CE7506AFE
:10129000083800F029F962E6D1F89400083800F027
:1012A00023F9B0E6D1F88C00083800F01DF9A4E667
:1012B000D1F88400083800F017F998E6C86F0838AC
:1012C00000F012F98DE6486F083800F00DF982E65B
:1012D000C86E083800F008F977E6486E083800F064
:1012E00003F96CE6C86D083800F0FEF861E6486D59
:1012F000083800F0F9F856E6C86C083800F0F4F841
:101300004BE6486C083800F0EFF840E6C86B083848
:1013100000F0EAF835E6486B083800F0E5F82AE610
:10132000C86A083800F0E0F81FE62A78C9F82800F3
:1013300001322A70C3E62A78C9F8200001322A70E7
:101340005AE72A78C9F8880001322A70DCE62A7840
:10135000C4F8800001322A708EE72A78C9F8680044
:1013600001322A70C3E62A78C8F8600001322A7078
:1013700014E72A78C9F8480001322A70ABE62A78C7
:10138000C8F8400001322A701FE740298E4628BF66
:101390004FF0400E02EB0E0302930123CEEB01014E
:1013A0004FEA0E4800250193BCE600BF88004000CC
:1013B000C80040002DE9F04100F03AFD2F4C304BC1
:1013C0003048DFF8D880304F304D314EDFF8D0C094
:1013D000DFF8D0E000221A605A609A60DA601A6181
:1013E0005A619A61DA611A625A629A62DA621A631F
:1013F0005A639A63DA631A645A649A64DA641A65FF
:101400005A659A65DA651A665A669A66DA661A67DE
:101410005A679A67DA67C3F880202168C3F8842086
:1014200041F480212160016841F040710160C3F303
:10143000072188F8001004F52834C3F307411B0E78
:101440003970CC342B7000F12040FF238CF8003031
:10145000104D8EF8003000F6041033700E49012351
:1014600008F8083C702622704FF40014102207F888
:101470002C3C2E7004600A70BDE8F081348004407A
:101480000000FF1F00D80040B0200740B4200740F4
:101490001020074035E400E0082107409C20074069
:1014A000802007408820074072B60D480268B2FAD3
:1014B00082F30B2B10DC4FF00041D94022EA0102ED
:1014C000026062B6074803EBC303DB00C2180021C9
:1014D000C15010465160704762B60020704700BF8F
:1014E0003007FF1FD003FF1F0D4B0E4AC31AA2FB8C
:1014F00003231B090B2B0CD80B4A127852B972B676
:101500000A484FF00041026821FA03F31A430260CF
:1015100062B67047064A1278002AF0D0FFF760B929
:10152000D003FF1F398EE338550DFF1F3007FF1F13
:10153000600DFF1F38B5164D2868E0B1018844885A
:10154000A14213DD03191B7A83B104F10803C21809
:101550000C1B002302E012F8011F21B10133A3424A
:10156000F9D1204638BD1C46204638BDFFF7BCFFE8
:101570000020286038BD074B1B780BB9002038BD10
:101580000220FFF70FF928600028D7D1F6E700BF47
:10159000700DFF1F600DFF1F0D4B1B78BBB910B501
:1015A0000C4C216803F0FF024B883F2B07DC07330C
:1015B0000B4401F1470003F8012F8342FBD1402384
:1015C0000B800120FFF770F90023236010BD7047E6
:1015D000680DFF1F6C0DFF1F08B5FEF747FFFEF7F4
:1015E00049FF00F001F8FAE738B52C4C237803B135
:1015F00038BD01232370FFF79DFF002842D100F082
:10160000F5F800283BD100F087F9002834D100F02C
:1016100019FA70BB00F092FA40BB00F00BFB10BB54
:1016200000F084FBE0B900232370EFF30583002B67
:10163000DED1EFF3108172B6194B186828B3194C3C
:10164000227812BB45691D60012323700DB3AA6186
:1016500001B962B600254577836898472570C7E7CA
:1016600000F028FDDFE700F023FDD9E700F01EFDC4
:10167000D3E700F019FDCDE700F014FDC7E700F057
:101680000FFDC0E700F018FDB9E70029B0D162B640
:1016900038BD054B1D600029DCD1DAE7750DFF1F51
:1016A0008810FF1F8C10FF1F8410FF1F30B42948C3
:1016B000294A2A4B2A4D6024E121047011701B78BD
:1016C000284C082B30D00A2B2748284937D00C2B20
:1016D0000CBF35223D2212232A60236002600B607A
:1016E000234B24491B78244ABBB101230B601360B0
:1016F000224B23491B78234A012B26D9042B0FD9CF
:10170000082B1ED9102B94BF862387230B601360F0
:101710001D4B01221A7030BC70470B601360E7E765
:1017200084230B601360F3E700F58E200F49083027
:10173000012213232A60236002600B60D0E7392264
:10174000F7E785230B601360E2E780230B601360EB
:10175000DEE700BF00400740014007403407FF1F9D
:1017600008B003400CB0034008B00B400CB00B4075
:10177000770DFF1F20B0034020B00B403507FF1F3F
:1017800024B0034024B00B40760DFF1F08B5104C69
:1017900008E0236859050DD423681A050FD423687F
:1017A000DB0411D423685803F3D5FFF7BFF823688F
:1017B0005905F1D500F02AF823681A05EFD500F095
:1017C000BBF82368DB04EDD500F04CF9EAE700BF75
:1017D0003480044008B5FFF7D9FF00BF014B102249
:1017E0001A80704700200540704700BF054A064B2D
:1017F00010781B78C0B2DBB2984238BF4030C01AB4
:10180000704700BF7C0DFF1F7D0DFF1FF0B4384BEC
:101810001A7912F0300F2CD072B6997D01F0FF02C8
:1018200000293DD062B6334F334938780D78334EB6
:101830001C46C0B2EDB2431C402BE17928BF002307
:10184000AB4202F1FF32C9B21CBFF154184612F08C
:10185000FF02F0D12A4B1B68C2B23A704BB1A842CA
:1018600036BFC5F14005401B40192728C4BF0122DF
:101870001A701F49CA78D2B2150616D452060DD571
:101880001B4B1B795B0609D51E4B1F491B680022A9
:101890000A7003B11A70164B3C22DA70F0BC704724
:1018A0004022D9795A7462B6E3E70B791C06E5D574
:1018B000164B174E1C783378E4B2DBB29C420ED044
:1018C000144D01E0A3420AD00133402B28BF00236E
:1018D0000879E85CC0B2C871087D0728F2D9DBB28C
:1018E000034933700B79180644BF7C23CB70C5E7DE
:1018F00000A006407C0DFF1F7D0DFF1FC00DFF1FC8
:10190000780DFF1F040EFF1F000EFF1F080EFF1FA4
:10191000010EFF1F800DFF1F054A064B10781B7834
:10192000C0B2DBB2984238BF4030C01A704700BF27
:101930007C0EFF1F110EFF1FF0B4384B1A7912F006
:10194000300F2CD072B6997D01F0FF0200293DD0F6
:1019500062B6334F334938780D78334E1C46C0B2E7
:10196000EDB2431C402BE17928BF0023AB4202F1CA
:10197000FF32C9B21CBFF154184612F0FF02F0D179
:101980002A4B1B68C2B23A704BB1A84236BFC5F1B0
:101990004005401B40192728C4BF01221A701F4967
:1019A000CA78D2B2150616D452060DD51B4B1B7938
:1019B0005B0609D51E4B1F491B6800220A7003B144
:1019C0001A70164B3C22DA70F0BC70474022D9796D
:1019D0005A7462B6E3E70B791C06E5D5164B174E31
:1019E0001C783378E4B2DBB29C420ED0144D01E097
:1019F000A3420AD00133282B28BF00230879E85CD2
:101A0000C0B2C871087D0728F2D9DBB20349337030
:101A10000B79180644BF7C23CB70C5E700B00640A5
:101A20007C0EFF1F110EFF1F3C0EFF1F0C0EFF1F31
:101A3000800EFF1F100EFF1F840EFF1F7D0EFF1F65
:101A4000140EFF1F054A064B10781B78C0B2DBB29C
:101A5000984238BF4030C01A704700BF8C0EFF1F3D
:101A60008D0EFF1F30B42B4B1A7994061FD52A48D0
:101A7000DA790378294901333F2B0978C8BF00235D
:101A80008B42D2B203D0264CD9B2E2540170254A1F
:101A9000116861B1244A1278D2B2934236BFC2F1C2
:101AA00040029B1A9B18272BC4BF01230B70194AB5
:101AB000D378DBB2180611D45A060DD5154B1B7915
:101AC0005B0609D5194B1A491B6800220A7003B13D
:101AD0001A70104B2C22DA7030BC7047117909064D
:101AE000EAD5144910480C780178C9B28C420DD05F
:101AF0004A1C272A84BF00210A460F4D054C98BF77
:101B0000D1B2AA5CD2B2E2710170D5E76C21D1707A
:101B1000D2E700BF00C006408C0EFF1F8D0EFF1FD6
:101B2000B80EFF1F880EFF1FF90EFF1FFC0EFF1FD0
:101B3000F80EFF1F000FFF1F900EFF1F054A064BF8
:101B400010781B78C0B2DBB2984238BF4030C01A60
:101B5000704700BF080FFF1F090FFF1F30B42B4B4A
:101B60001A7994061FD52A48DA790378294901336E
:101B70003F2B0978C8BF00238B42D2B203D0264C3A
:101B8000D9B2E2540170254A116861B1244A127831
:101B9000D2B2934236BFC2F140029B1A9B18272B48
:101BA000C4BF01230B70194AD378DBB2180611D4D5
:101BB0005A060DD5154B1B795B0609D5194B1A49E9
:101BC0001B6800220A7003B11A70104B2C22DA70C5
:101BD00030BC704711790906EAD5144910480C78D1
:101BE0000178C9B28C420DD04A1C272A84BF00213B
:101BF0000A460F4D054C98BFD1B2AA5CD2B2E27131
:101C00000170D5E76C21D170D2E700BF00D006404B
:101C1000080FFF1F090FFF1F340FFF1F040FFF1FC7
:101C2000750FFF1F780FFF1F740FFF1F7C0FFF1F23
:101C30000C0FFF1F054A064B10781B78C0B2DBB2B1
:101C4000984238BF4030C01A704700BF840FFF1F52
:101C5000850FFF1F30B42B4B1A7994061FD52A48E5
:101C6000DA790378294901333F2B0978C8BF00236B
:101C70008B42D2B203D0264CD9B2E2540170254A2D
:101C8000116861B1244A1278D2B2934236BFC2F1D0
:101C900040029B1A9B18272BC4BF01230B70194AC3
:101CA000D378DBB2180611D45A060DD5154B1B7923
:101CB0005B0609D5194B1A491B6800220A7003B14B
:101CC0001A70104B2C22DA7030BC7047117909065B
:101CD000EAD5144910480C780178C9B28C420DD06D
:101CE0004A1C272A84BF00210A460F4D054C98BF85
:101CF000D1B2AA5CD2B2E2710170D5E76C21D17089
:101D0000D2E700BF00A00E40840FFF1F850FFF1F0A
:101D1000B00FFF1F800FFF1FF10FFF1FF40FFF1FFA
:101D2000F00FFF1FF80FFF1F880FFF1F054A064B1C
:101D300010781B78C0B2DBB2984238BF4030C01A6E
:101D4000704700BF0010FF1F0110FF1F30B42C4B65
:101D50005A6894021FD52B48DA6803782A49013360
:101D60003F2B0978C8BF00238B4204D0274CD2B246
:101D7000D9B2E2540170264A116861B1254A12783D
:101D8000D2B2934236BFC2F140029B1A9B18272B56
:101D9000C4BF01230B701A4A9368180202D5526817
:101DA000110211D45A020DD5154B5B685B0209D59F
:101DB000194B1A491B6800220A7003B11A70184B9C
:101DC00000221A6030BC7047164A124910780A780F
:101DD000D2B290420DD00132272A84BF00200246A1
:101DE000114D074C98BFD0B2AA5CD2B2E260087025
:101DF000D8E70E480A4A0024012104601160D1E7A7
:101E000000400C400010FF1F0110FF1F2C10FF1F8F
:101E1000FC0FFF1F6D10FF1F7010FF1F6C10FF1FC6
:101E2000580188437410FF1F0410FF1F5C01884392
:101E300072B6184A184B19491160702280211A7025
:101E40001A46197013781B06FCD510B5144B84B0D4
:101E5000186862B6134B144C984298BF00EB800090
:101E600001A998BF40000A2200F028F901A92046E4
:101E7000002311F8012B01333AB10A2B20F8022F6D
:101E8000F7D11623237004B010BD5B00DBB22370C2
:101E900004B010BD040002400000024000000741F1
:101EA0000C0002407F9698001C08FF1F10B4EFF34F
:101EB000108272B6437F33B9017F012908D003290C
:101EC00010D00123437702B962B65DF8044B704726
:101ED000114C2168A1B1114943610B68836108600D
:101EE0005861EEE70E4C216881B10E4943610B68E1
:101EF0008361086058610C4B4FF080511960E0E736
:101F0000064B4161816120601860DAE7054B416151
:101F1000816120601860EEE78810FF1F8410FF1FAA
:101F20007810FF1F7C10FF1F04ED00E010B4047F49
:101F30004160022CC26003D05DF8044BFFF7B6BFCE
:101F400083685DF8044B184770B5EFF3108272B6E2
:101F50000C4C206880B10C4E00254369236073B19E
:101F60009D6102B962B6457783689847EFF31082A6
:101F700072B620680028F0D102B962B670BD336035
:101F8000EFE700BF7810FF1F7C10FF1FFFF7DCBFDB
:101F9000184A30B41468002C27D0036821688B429B
:101FA0000ED2CB1A00218460C1602360E060106013
:101FB0000223037530BC704711688B42144608D366
:101FC000A2685B1A0360002AF6D18260C460A06038
:101FD000EEE7D268C2608460E060C568CB1A022276
:101FE000A8602360027530BC70478460C4601060D4
:101FF000DEE700BF8010FF1FF8B5224E34682CB317
:102000002368002B3AD1204F1D4604E03468ECB120
:102010002368002B32D1A36803B1DD6020693360EF
:10202000036825751B68BB4221D1037F4560022BE5
:10203000C46020D0FFF73AFF6368002BE6D023602E
:102040002046FFF7A5FF3468002CE1D1EFF31083A1
:1020500072B60E4A00211068116003B962B628B149
:102060008468FFF795FF20460028F9D1F8BD224685
:1020700000219847E0E783689847DDE7013B23604C
:10208000E4E700BF8010FF1F2D1F00009010FF1F0E
:10209000024A136801331360FFF7AEBF7C0CFF1FC9
:1020A000704700BF704700BF704700BF704700BF58
:1020B000704700BF704700BF704700BFF0B44D1EAF
:1020C0002E46002400E00134B0FBF2F302FB1300C3
:1020D000092800F130078ABF3730F8B2C0B206F8DD
:1020E000010F1846002BEED10A1953704CB110782D
:1020F00015F8016F28700133E01A834202F8016974
:10210000F5DB0846F0BC704770B50F4E0F4D761BDF
:10211000B61018BF002405D0013455F8043B984789
:10212000A642F9D10A4E0B4D761B00F0D1F9B6103C
:1021300018BF002406D0013455F8043B9847A64246
:10214000F9D170BD70BD00BFDC240000DC240000AC
:10215000E4240000DC240000024B13B1024800F02C
:1021600005B87047000000007921000000230146F7
:102170001A46184600F014B838B5074D074C2C1B0A
:10218000A41005D0013C55F8043D9847002CF9D126
:10219000BDE8384000F0A6B90000000000000000D3
:1021A0002DE9F047254C2568D5F848410646884674
:1021B00092469946C4B360681F2817DC431C76B169
:1021C00004EB80050122C5F888A0D4F8881182406C
:1021D0001143022EC4F88811C5F808911ED00230B0
:1021E000636044F820800020BDE8F087144B03B3FF
:1021F0004FF4C870AFF300800446D0B1D5F8483131
:10220000002780E88800C5F8484138460123C4F813
:102210008871C4F88C71002EE1D0D1E7D4F88C110C
:102220000A43C4F88C21DAE705F5A674C5F84841DD
:10223000C1E74FF0FF30BDE8F08700BFCC240000BD
:10224000000000004008FE4340A004404408FE4354
:1022500044A004400018FE4300C004403000FE4388
:10226000309004403400FE43349004401C18FE4378
:102270001CC004401018FE4310C004400818FE4360
:1022800008C004400C18FE430CC004400C10FE4370
:102290000CB004401010FE4310B004401810FE4370
:1022A00018B004401C10FE431CB004401410FE4340
:1022B00014B004400418FE4304C004400010FE4360
:1022C00000B004400008FE4300A004400408FE43A0
:1022D00004A004400C08FE430CA004400808FE4380
:1022E00008A004401418FE4314C004401818FE430C
:1022F00018C004400410FE4304B004400810FE431C
:1023000008B004406820FE4368D004401400FE4337
:10231000149004403800FE43389004403C00FE43D3
:102320003C9004404000FE43409004404808FE4377
:1023300048A004404C08FE434CA004402808FE433B
:1023400028A004402C08FE432CA004406020FE433B
:1023500060D004406420FE4364D004402010FE435B
:1023600020B004402410FE4324B004402810FE4353
:1023700028B004402C10FE432CB004404400FE431F
:10238000449004407000FE43709004407400FE438B
:10239000749004406800FE43689004405008FE4377
:1023A00050A004405808FE4358A004405C08FE4377
:1023B0005CA004405408FE4354A004402018FE438F
:1023C00020C004402418FE4324C004401008FE43EB
:1023D00010A004401408FE4314A004403818FE4323
:1023E00038C004403418FE4334C004403018FE4363
:1023F00030C004403C18FE433CC004402C18FE434F
:102400002CC004402820FE4328D004402C20FE434A
:102410002CD004400020FE4300D004400420FE43A2
:1024200004D004400820FE4308D004400C20FE43A2
:102430000CD004401020FE4310D004401420FE4372
:1024400014D0044015191519000100003807FF1FAA
:1024500012000000000200006407FF1F4900000096
:1024600000220100B007FF1F210000000021010031
:102470009607FF1F0900000000220000D407FF1F7D
:102480001C000000002100007607FF1F090000006B
:10249000000300001808FF1F0000000001030904EA
:1024A0004C07FF1F0000000002030904F007FF1F94
:1024B00000000000030309041C08FF1F00000000C7
:1024C0000000000000000000000000003808FF1FAE
:1024D000F8B500BFF8BC08BC9E4670475921000003
:0424E00035040000BF
:0424E400F8B500BF88
:1024E800FFFFFFFF0A040000120110010000004076
:1024F800C016860477020102030100001803540085
:10250800650065006E00730079006400750069005D
:102518006E006F0009024900020100C03209040080
:10252800000203000000092111010001221C00071C
:102538000583034000010705040340000109040165
:1025480000020300000009211101000122210007F7
:102558000581034000010705020320000200000076
:1025680006C9FF0904A15C7508150026FF009540FF
:102578000975810295200976910295040976B102C0
:10258800C000000006ABFF0A0002A1017508150093
:1025980026FF00954009018102954009029102C079
:1025A80026035400650065006E007300790064001E
:1025B800750069006E006F0020005200610077000E
:1025C8004800490044000000040309040C0300000B
:1025D80000000000000000000000000000000000F3
:1025E800000000000000000000000000240BFF1F96
:1025F8008C0BFF1FF40BFF1F000000000000000001
:1026080000000000000000000000000000000000C2
:1026180000000000000000000000000000000000B2
:1026280000000000000000000000000000000000A2
:102638000000000000000000000000000000000092
:102648000000000000000000000000000000000082
:102658000000000000000000000000000000000072
:102668000000000000000000000000000000000062
:102678000000000000000000000000000000000052
:102688000000000000000000000000000000000042
:1026980001000000000000000E33CDAB34126DE6DF
:1026A800ECDE05000B000000000000000000000048
:1026B8000000000000000000000000000000000012
:1026C8000000000000000000000000000000000002
:1026D80000000000000000000000000000000000F2
:1026E80000000000000000000000000000000000E2
:00000001FF
